:1000000010C02AC029C028C027C026C025C024C0CF
:1000100023C022C021C020C01FC01EC01DC01CC0E4
:100020001BC011241FBECFE5D1E0DEBFCDBF10E065
:10003000A0E6B0E0EEE9F3E002C005900D92A03733
:10004000B107D9F720E0A0E7B0E001C01D92AE38BB
:10005000B207E1F701D1A1C1D3CFDC01FA011082CF
:100060008C918623E9F78CE18A95F1F7000088E30B
:100070008A95F1F700C08C91862319F08081816008
:10008000808388E38A95F1F700C08C91862319F06C
:1000900080818260808388E38A95F1F700C08C912B
:1000A000862319F080818460808388E38A95F1F744
:1000B00000C08C91862319F080818860808388E35A
:1000C0008A95F1F700C08C91862319F080818061B8
:1000D000808388E38A95F1F700C08C91862319F01C
:1000E00080818062808388E38A95F1F700C08C91DB
:1000F000862319F080818064808388E38A95F1F7F4
:1001000000C08C91862319F080818068808388E309
:100110008A95F1F700C08CE18A95F1F70000089507
:10012000FC019081862F80959823908398E39A957F
:10013000F1F700C0908140FF02C0962B01C09823C8
:10014000908398E39A95F1F700C0908141FF02C037
:10015000962B01C09823908398E39A95F1F700C0FD
:10016000908142FF02C0962B01C09823908398E3B0
:100170009A95F1F700C0908143FF02C0962B01C011
:100180009823908398E39A95F1F700C0908144FFFB
:1001900002C0962B01C09823908398E39A95F1F7BB
:1001A00000C0908145FF02C0962B01C09823908328
:1001B00098E39A95F1F700C0908146FF02C0962B14
:1001C00001C09823908398E39A95F1F700C047FF08
:1001D00004C08081862B808303C090819823908304
:1001E00088E38A95F1F700C08081862B808398E3AD
:1001F0009A95F1F700C088E38A95F1F700C0089559
:10020000FF920F931F93CF93DF938C01F62EEA0199
:1002100010928D0010928C00E0918C00F0918D0076
:10022000EC0FFD1F40816F2DC8017ADF20918C00FB
:1002300030918D002F5F3F4F30938D0020938C00C5
:10024000FE01E20FF31F80818111E6CFDF91CF9194
:100250001F910F91FF90089580E886BD16BCD49A37
:10026000D39AD29A8BB38BBB8BB38BBB8BB38BBB29
:1002700087B387BBC29AD99AD19A94E088E020E1EB
:1002800034E148E15CE1B29B51C01BBA6FE372E418
:10029000EFE061507040E040E1F700C000009BBB20
:1002A0006FE372E4EFE061507040E040E1F700C0BE
:1002B00000008BBB6FE372E4EFE061507040E04000
:1002C000E1F700C000008BBB6FE372E4EFE0615028
:1002D0007040E040E1F700C000002BBB6FE372E428
:1002E000EFE061507040E040E1F700C000003BBB30
:1002F0006FE372E4EFE061507040E040E1F700C06E
:1003000000004BBB6FE372E4EFE061507040E040EF
:10031000E1F700C000005BBB6FE372E4EFE0615007
:100320007040E040E1F700C00000ADCF10928B00BC
:1003300010928A0049E850E061E089E390E08DDEA8
:1003400040E650E062E08BE390E05ADF20918A00C3
:1003500030918B00C901019690938B0080938A00A5
:10036000F901E059FF4F409189004083489721F4FB
:1003700010928B0010928A0040E750E062E08BE31D
:1003800090E03EDF42E262E08BE390E0C9DE4AE0CB
:0E03900062E08BE390E0C4DECDCFF894FFCFA7
:10039E0054686520636F6465206973206F6B22005B
:00000001FF
